:100000002AC044C043C042C041C040C03FC03EC0FF
:100010003DC03CC03BC03AC039C038C047C036C004
:1000200035C034C033C000000000000000001010D4
:1000300010101010100018181818181818001C1C90
:100040001C1C1C1C1C001E1E1E1E1E1E1E001F1F14
:100050001F1F1F1F1F0011241FBECFE5D4E0DEBFEE
:10006000CDBF10E0A0E6B0E0EEE7FAE002C00590F8
:100070000D92A438B107D9F710E0A4E8B0E001C0B0
:100080001D92AA38B107E1F725D0F7C4B9CF8FEF99
:1000900081BB12BA14BA15BA86B18E6886B987B117
:1000A000806C87B9C5D141D1789408951F920F9281
:1000B0000FB60F9211248F939F9384B195B19093B3
:1000C0008500809384009F918F910F900FBE0F90B9
:1000D0001F901895AF92BF92CF92DF92EF92FF924E
:1000E0000F931F93CF93DF93D2DF83E060E04DD176
:1000F00080E690E06BE025D180E090E0CCE3D0E0BA
:100100000BE610E00F2EFCE7EF2EF0E0FF2EF02DB7
:100110000F2EF1E8CF2EF0E0DF2EF02DAA24BB2425
:1001200016C0369AEFE1FEE43197F1F700C0000007
:100130004091880050918900209184003091850081
:10014000240F351F309389002093880001968C334B
:1001500091053CF38091880090918900BE0166D49E
:100160007093890060938800F1E064307F0798F411
:1001700080E090E06AD32AE037ED43E25BE3F3D31B
:100180002AE037ED43E25CE3CCD233D370938700AF
:100190006093860058C09B012550314041E02F38C4
:1001A0003407C0F480E090E050D32AE037ED43E21A
:1001B0005BE3D9D321EE3AE744E15FE34DD22CE68D
:1001C00039E049E75BE3ADD214D3709387006093C5
:1001D000860039C09B012559324025393105C0F4CC
:1001E00080E090E032D32AE037ED43E25BE3BBD31B
:1001F00023E333E343EB5FE32FD22FE632E143E81F
:100200005AE38FD2F6D270938700609386001BC0AA
:10021000E3E06B327E07B8F080E090E016D32AE08E
:1002200037ED43E25BE39FD326E636E646EE5FE337
:1002300013D222E539E44DE959E373D2DAD270934F
:1002400087006093860071D080E060E09ED0C80196
:1002500060E177D082E061E098D0C70164E071D0BE
:1002600086E061E092D0809186009091870064E002
:10027000C2D18CE061E089D0C60162E062D0C501E4
:1002800066CF982F907F92BB909A929AE9EFF0E018
:100290003197F1F700C0000092989098E9EFF0E0F4
:1002A0003197F1F700C0000090E082959295907F21
:1002B0009827807F982782BB909A929A89EF90E046
:1002C0000197F1F700C0000092989098E9EFF0E0F4
:1002D0003197F1F700C000000895982F907F92BBEE
:1002E000929AE9EFF0E03197F1F700C000009298A0
:1002F000E9EFF0E03197F1F700C0000090E082955F
:100300009295907F9827807F982782BB929A89EF59
:1003100090E00197F1F700C000009298E9EFF0E05B
:100320003197F1F700C00000089583EC99E0019740
:10033000F1F700C0000081E0D0DF089582E0CDDF5A
:100340000895EF92FF920F931F93CF93DF93162F91
:100350000097A1F0662391F0082FE82EE7017E01B7
:10036000F92EE70183EC99E00197F1F700C0000056
:10037000899187DF7E01E01AE116A0F3DF91CF912A
:100380001F910F91FF90EF900895623031F063302C
:1003900031F0613029F4805C03C08C5E01C08C5A5E
:1003A000E3ECF9E03197F1F700C00000806895DFD9
:1003B00008951F93CF93DF93EC01862F642FE5DF21
:1003C000CE01FE012491222361F010E0FC01849112
:1003D00058DF1F5FCE01810F911DFC012491222364
:1003E000A9F7DF91CF911F910895EF92FF920F939C
:1003F0001F93CF93DF937C01062F000F000F000F98
:100400000064C0E0D0E0F701EC0FFD1F14919E01E5
:10041000200F822F62DF812F34DF2196C830D10573
:1004200091F7DF91CF911F910F91FF90EF90089579
:10043000CF93DF9385EA9EE00197F1F700C00000BB
:1004400012BA12BA81B3806F81BB81B3876081BB5E
:1004500080E382BB929AE9EFF0E03197F1F700C0B8
:1004600000009298E9EFF0E03197F1F700C000004A
:1004700082BB929A89EF90E00197F1F700C00000EB
:100480009298E9EFF0E03197F1F700C0000080E2C8
:1004900082BB929A89EF90E00197F1F700C00000CB
:1004A0009298E9EFF0E03197F1F700C0000088E2A0
:1004B00014DF8CE012DFC0E0D0E0CE01880F991F7E
:1004C000880F991F880F991F8A5D9F4F6C2F8DDFB2
:1004D0002196C830D10589F7DF91CF9108950F9308
:1004E0001F93082F882331F010E08EE1F6DE1F5FA6
:1004F0001017D8F31F910F9108950F931F93082F92
:10050000882331F010E088E1E8DE1F5F1017D8F390
:100510001F910F9108958EE0E0DE08958FE0DDDEFB
:1005200008958CE0DADE089588E0D7DE08958CE047
:10053000D4DE08950F931F93082F882331F010E025
:1005400080E1CBDE1F5F1017D8F31F910F91089544
:100550000F931F93082F882331F010E084E1BDDE54
:100560001F5F1017D8F31F910F910895BF92CF927C
:10057000DF92EF92FF920F931F93CF93DF93042F9D
:1005800046E0849FA0011124202F30E0429FC0014B
:10059000439F900D529F900D112470E05BD27B0120
:1005A0000023F9F0CB0166E070E040D2C0E0D0E07B
:1005B00010E00F2EF5E0DF2EF02DCC24B82ECE016A
:1005C0000596E816F90628F4EC16FD0620F08B2DAA
:1005D00003C08D2D01C08C2D54DE1F5F2696101791
:1005E00070F3DF91CF911F910F91FF90EF90DF900B
:1005F000CF90BF900895CF93DF93EC016230C9F0A4
:10060000633018F4613029F51EC0633041F0643066
:1006100001F568EE73E00AD2862F805D32DECE01EE
:1006200064E670E003D2CB016AE070E0FFD1805D48
:1006300028DE2AE030E0CE01B901F8D1CB01B901C2
:10064000F5D1805D1EDECE016AE070E0EFD1805D05
:1006500018DEDF91CF9108955058BB27AA270ED0FE
:1006600048C139D130F03ED120F031F49F3F11F430
:100670001EF42EC10EF4E095E7FB24C1E92F4AD108
:1006800080F3BA17620773078407950718F071F4AF
:100690009EF562C10EF4E0950B2EBA2FA02D0B0132
:1006A000B90190010C01CA01A0011124FF27591BB7
:1006B00099F0593F50F4503E68F11A16F040A22FBD
:1006C000232F342F4427585FF3CF4695379527952E
:1006D000A795F0405395C9F77EF41F16BA0B620B2D
:1006E000730B840BBAF09150A1F0FF0FBB1F661F74
:1006F000771F881FC2F70EC0BA0F621F731F841FB7
:1007000048F4879577956795B795F7959E3F08F0DC
:10071000B3CF9395880F08F09927EE0F979587959B
:1007200008950CD0E6C0DED040F0D5D030F021F4F2
:100730005F3F19F0C7C0511110C1CAC0EBD098F388
:100740009923C9F35523B1F3951B550BBB27AA2752
:1007500062177307840738F09F5F5F4F220F331FC4
:10076000441FAA1FA9F333D00E2E3AF0E0E830D090
:1007700091505040E695001CCAF729D0FE2F27D093
:10078000660F771F881FBB1F261737074807AB0761
:10079000B0E809F0BB0B802DBF01FF2793585F4FD6
:1007A0002AF09E3F510568F08DC0D7C05F3FECF343
:1007B000983EDCF3869577956795B795F7959F5F9B
:1007C000C9F7880F911D9695879597F90895E1E0EF
:1007D000660F771F881FBB1F621773078407BA074E
:1007E00020F0621B730B840BBA0BEE1F88F7E095A9
:1007F000089598D088F09F5790F0B92F9927B75156
:10080000A0F0D1F0660F771F881F991F1AF0BA95D4
:10081000C9F712C0B13081F09FD0B1E008959CC0FB
:10082000672F782F8827B85F39F0B93FCCF38695CA
:1008300077956795B395D9F73EF490958095709527
:1008400061957F4F8F4F9F4F0895E89409C097FBA4
:100850003EF490958095709561957F4F8F4F9F4F97
:100860009923A9F0F92F96E9BB279395F6958795DB
:1008700077956795B795F111F8CFFAF4BB0F11F49E
:1008800060FF1BC06F5F7F4F8F4F9F4F16C0882345
:1008900011F096E911C0772321F09EE8872F762F7B
:1008A00005C0662371F096E8862F70E060E02AF0BC
:1008B0009A95660F771F881FDAF7880F96958795A8
:1008C00097F9089597F99F6780E870E060E00895D0
:1008D0009FEF80EC089500240A9416161706180658
:1008E0000906089500240A94121613061406050634
:1008F0000895092E0394000C11F4882352F0BB0FC5
:1009000040F4BF2B11F460FF04C06F5F7F4F8F4F27
:100910009F4F089557FD9058440F551F59F05F3F62
:1009200071F04795880F97FB991F61F09F3F79F011
:1009300087950895121613061406551FF2CF469593
:10094000F1DF08C0161617061806991FF1CF869515
:100950007105610508940895E894BB2766277727F9
:10096000CB0197F908950BD0C4CFB5DF28F0BADFDB
:1009700018F0952309F0A6CFABCF1124EECFCADF34
:10098000A0F3959FD1F3950F50E0551F629FF001A2
:10099000729FBB27F00DB11D639FAA27F00DB11DFB
:1009A000AA1F649F6627B00DA11D661F829F222784
:1009B000B00DA11D621F739FB00DA11D621F839F0B
:1009C000A00D611D221F749F3327A00D611D231FE1
:1009D000849F600D211D822F762F6A2F11249F572F
:1009E00050408AF0E1F088234AF0EE0FFF1FBB1F52
:1009F000661F771F881F91505040A9F79E3F5105F1
:100A000070F060CFAACF5F3FECF3983EDCF38695A1
:100A100077956795B795F795E7959F5FC1F7FE2B9B
:100A2000880F911D9695879597F90895AA1BBB1B72
:100A300051E107C0AA1FBB1FA617B70710F0A61BDE
:100A4000B70B881F991F5A95A9F780959095BC01FF
:100A5000CD01089597FB092E07260AD077FD04D013
:100A6000E5DF06D000201AF4709561957F4F089558
:0E0A7000F6F7909581959F4F0895F894FFCF6B
:100A7E002E4C4F4144494E472E2E002E4469676935
:100A8E00742E204C75784D657465720045203D209E
:040A9E00006C780070
:00000001FF
